:020000040800F2
:100000003804002005010008C1030008950200081B
:10001000BD03000871010008470A00080000000045
:10002000000000000000000000000000950600082D
:1000300075010008000000009D050008A9070008E0
:100040001F0100081F0100081F0100081F01000810
:100050001F0100081F0100081F0100081F01000800
:100060001F0100081F0100081F0100081F010008F0
:100070001F0100081F0100081F0100081F010008E0
:100080001F0100081F0100081F0100081F010008D0
:100090001F0100081F0100081F0100081F010008C0
:1000A0001F0100081F0100081F0100081F010008B0
:1000B0001F0100081F0100081F0100081F010008A0
:1000C0001F0100081F0100081F0100081F01000890
:1000D0001F0100080D0800081F0100081F0100088B
:1000E0001F0100081F0100081F010008DFF810D0E1
:1000F00000F02CF800480047050C0008AFF3008022
:10010000380400200648804706480047FEE7FEE71F
:10011000FEE7FEE7FEE7FEE7FEE7FEE7FEE7FEE7B7
:10012000AD070008ED000008D2B201E000F8012B95
:10013000491EFBD270470022F6E710B513460A4667
:1001400004461946FFF7F0FF204610BD064C074D48
:1001500006E0E06840F0010394E807009847103497
:10016000AC42F6D3FFF7C6FFE812000808130008F8
:1001700000BFFEE770472DE9F0410246002500264A
:10018000002000230024002791F803C00CF00F0585
:1001900091F803C00CF0100CBCF1000F03D091F8E3
:1001A00002C04CEA050591F800C0BCF1000F31D047
:1001B000146800202BE04FF0010C0CFA00F3B1F8AA
:1001C00000C00CEA03069E4220D183004FF00F0CC2
:1001D0000CFA03F7BC4305FA03FC4CEA040491F85B
:1001E00003C0BCF1280F06D14FF0010C0CFA00FC43
:1001F000C2F814C00AE091F803C0BCF1480F05D161
:100200004FF0010C0CFA00FCC2F810C0401C08288A
:10021000D1D31460B1F800C0BCF1FF0F34DD5468D5
:1002200000202EE000F1080C4FF0010808FA0CF352
:10023000B1F800C00CEA03069E4221D183004FF0C2
:100240000F0C0CFA03F7BC4305FA03FC4CEA040458
:1002500091F803C0BCF1280F05D100F1080C08FA91
:100260000CF8C2F8148091F803C0BCF1480F07D114
:1002700000F1080C4FF0010808FA0CF8C2F81080E1
:10028000401C0828CED35460BDE8F081416170471E
:100290000161704700BFFEE770B5024600240025EB
:1002A00000230020958A138B1B0445EA030626F0E1
:1002B0007F4404EA01068E4201D1012000E00020C3
:1002C00070BD21B1028842F48072028004E002888D
:1002D0004FF6FF631A400280704721B1028842F452
:1002E0000072028004E002884FF6FF531A40028039
:1002F00070470CB502460020002301930093009242
:100300000B0F019321F07F41019B1BB1009B143324
:10031000009303E0090C009B18330093009B1B68BB
:100320000B400BB1012000E000200CBD12B141F0E8
:10033000010102E04FF6FE7319400182704701820D
:100340007047000008B50121042000F029F91020B1
:10035000ADF800008DF8030003208DF80200694617
:100360000348FFF708FF10210148FFF791FF08BD80
:100370000008014010B5012005490860102105481A
:10038000FFF786FF4FF47A7000F008FC10BD000004
:10039000900121420008014010B500200549086085
:1003A00010210548FFF772FF4FF47A7000F0F6FB5A
:1003B00010BD0000900121420008014000BFFEE78F
:1003C0007047000070B5002100230F22C47804B3E9
:1003D000154C246804F4E064C4F5E064210AC1F11A
:1003E0000403CA40447804FA03F18478144021439A
:1003F00009010E4C0678A155047804F01F0501246C
:10040000AC4005786D11AD0005F1E025C5F800415F
:1004100009E0047804F01F050124AC40044D06787F
:10042000761145F8264070BD0CED00E000E400E0D8
:1004300080E100E070B504460D4600BF4FF4003186
:100440001C48FFF756FF0028F8D101211948FFF793
:1004500038FF00BF18491748FFF71EFF0028F9D0E2
:10046000002278211348FFF761FF00BF13491148AC
:10047000FFF712FF0028F9D021460E48FFF75FFF73
:1004800000BF0E49891C0B48FFF706FF0028F8D073
:1004900029460848FFF753FF00BF0849891C054853
:1004A000FFF7FAFE0028F8D001210248FFF715FFF8
:1004B00070BD0000005800400100030082000700EA
:1004C00070B505460C4645F0B00000F059F8102113
:1004D00041EA141000F054F804F00F0000F050F856
:1004E00070BD00002DE9F04105460E461746721E0C
:1004F000D206110E6A1E5206100EFFF7E1FF00240D
:1005000009E0A7F12001134A02EB0111085D00F098
:100510003EF8601CC4B2082CF3DB721ED206110E2A
:100520006A1E012303EB4202D0B2FFF7C9FF002489
:100530000BE0A7F12001074A02EB011204F10801C8
:10054000505C00F024F8601CC4B2082CF1DBBDE85C
:10055000F0810000F80C00082DE9F04107460E4636
:100560001546002407E02A5D3019C1B23846FFF76E
:10057000B9FF601CC4B2285D0028F4D1BDE8F08149
:1005800010B5044621460020FFF754FF10BD10B5FA
:10059000044621464020FFF74DFF10BD7047000084
:1005A00029B1064A92690243044B9A6104E0034A66
:1005B00092698243014B9A6170470000001002402B
:1005C00030B500210022002400232D4D6D6805F078
:1005D0000C0121B1042905D0082923D105E0294DBA
:1005E000056022E0274D05601FE0254D6D6805F48C
:1005F0007012234D6D6805F48034022505EB92429C
:100600001CB9214D554305600BE01D4D6D6805F487
:1006100000351DB11C4D5543056002E0194D554391
:10062000056002E0174D056000BF00BF144D6D6806
:1006300005F0F0010909154D6B5C0568DD4045606A
:100640000F4D6D6805F4E061090A104D6B5C45685B
:10065000DD4085600A4D6D6805F46051C90A0B4D97
:100660006B5C4568DD40C560054D6D6805F4404133
:10067000890B074D6B5CC568B5FBF3F5056130BDB3
:100680000010024000127A0000093D000000002026
:1006900010000020704710B500F002F810BD0000F7
:1006A0000CB50020019000903348006840F4803081
:1006B0003149086000BF3048006800F40030009005
:1006C0000198401C0190009818B90198B0F5A06FEE
:1006D000F1D12948006800F4003010B101200090E9
:1006E00001E0002000900098012843D123480068D1
:1006F00040F01000214908600846006820F003001F
:1007000008600846006840F0020008601A48406827
:10071000194948600846406848600846406840F407
:10072000806048600846406820F47C1048600846B5
:10073000406840F4E81048600846006840F0807067
:10074000086000BF0C48006800F000700028F9D075
:100750000948406820F0030007494860084640689F
:1007600040F00200486000BF0348406800F00C0001
:100770000828F9D10CBD0000001002400020024002
:10078000042808D14FF0E021096941F004014FF03D
:10079000E022116107E04FF0E021096921F0040136
:1007A0004FF0E022116170477047000010B5134808
:1007B000006840F00100114908600846406810498F
:1007C00008400E494860084600680E4908400B4939
:1007D00008600846006820F48020086008464068E9
:1007E00020F4FE0048604FF41F008860FFF753FFBD
:1007F0004FF000600449086010BD00000010024086
:100800000000FFF8FFFFF6FE08ED00E010B540F233
:1008100025511B4800F057F888B1194800F00EF92F
:10082000C1B2184802780078401C164B1870164860
:10083000815440F22551124800F02AF81FE040F29E
:1008400024410F4800F03FF8C8B100200E49087459
:100850000A4601210220FFF77FFE002009490870A7
:10086000202211210848FFF75FFC05480088C4B228
:100870000348001D0088C4B201200449087010BD5F
:10088000003801401D000020240000201800002036
:1008900010B50022002340F66A14A14200D100BF27
:1008A0000A1201249440A3B2DC43048010BD21B19C
:1008B000828942F40052828104E082894DF6FF73FE
:1008C0001A408281704770B502460024002300253B
:1008D000002040F66A16B14200D100BFC1F34215B4
:1008E00001F01F03012606FA03F3012D02D19689B8
:1008F000334006E0022D02D1168A334001E0968A89
:1009000033400C12012606FA04F41688344013B161
:100910000CB1012000E0002070BDF0B503460024BA
:1009200000260025002040F66A17B94200D100BF1A
:100930001846C1F3421401F01F06012707FA06F515
:10094000012C01D10C3004E0022C01D1103000E068
:1009500014301AB107682F43076002E00768AF43FD
:100960000760F0BD2DE9F04786B005460E4600242D
:10097000A24600BFA1460027B08900B100BF2F46A4
:100980002C8A4CF6FF700440F08804432C82AC891A
:100990004EF6F3100440B08831890843718908434A
:1009A0000443AC81AC8A4FF6FF400440B089044355
:1009B000AC8201A8FFF704FE1F48874202D1DDF890
:1009C00010A001E0DDF80CA0A88900F4004040B1BF
:1009D0000AEBCA0000EB0A1031684900B0FBF1F8DD
:1009E00007E00AEBCA0000EB0A1031688900B0FB8F
:1009F000F1F86420B8FBF0F004012009642101FB48
:100A00001089A88900F4004040B1322000EBC900F1
:100A1000B0FBF1F000F00700044308E0322000EBE7
:100A200009106421B0FBF1F000F00F0004432C81A9
:100A300006B0BDE8F0870000003801400146888814
:100A4000C0F30800704700BFFEE700000FB4054B7D
:100A500010B503A9044A029800F017F810BC5DF81D
:100A600014FB0000E90B00082000002002E008C889
:100A7000121F08C1002AFAD170477047002001E018
:100A800001C1121F002AFBD170472DE9F84F99468A
:100A9000924688460546002706E025280AD051469A
:100AA0004A4690476D1C7F1C28780028F5D13846AF
:100AB000BDE8F88F002315F8011F18462E2915D11F
:100AC00015F8011F04232A290DD06FF02F02297871
:100AD000A1F13004092C09D800EB800002EB4000A2
:100AE00008446D1CF3E758F8040B6D1C2A78002AA3
:100AF000DDD0632A07D0732A0FD0104651464A46EC
:100B000090477F1C2AE018F8042B8DF80020002164
:100B10008DF801106E46012103E058F8046B4FF088
:100B2000FF315A074FF0000401D409E0641C8442ED
:100B30000BDA8C42FADB325D002AF7D105E0641C47
:100B40008C42FCDB305D0028F9D1274404E016F824
:100B5000010B51464A469047641EF8D26D1CA3E72C
:100B600010B504466FF00400FFF70AFEE11704EB2E
:100B70005171C1F3C701074A11701046007800EBAC
:100B80004001C1EBC0104FF6FF7101EAC0000249FD
:100B9000088010BD14000020160000200146114AF4
:100BA00012884A434FF0E0235A6100229A611A46A4
:100BB000126942F001021A6100BF4FF0E022106991
:100BC00000F001021AB100F48032002AF5D04FF093
:100BD000E022126922F001024FF0E0231A610022A4
:100BE0009A6170471600002000BF054A128802F083
:100BF0004002002AF9D0C2B2014B1B1D1A80704777
:100C0000003801404820FFF7ABFFFFF79BFB4FF494
:100C1000E13000F019F80EE0FFF7BEFB4FF47A70F8
:100C2000FFF7BCFFFFF7A6FB4FF47A70FFF7B6FFA4
:100C300001A0FFF70BFFEFE73F3F3F3F313131317D
:100C4000313131313100000010B586B00446012148
:100C50000420FFF7A5FC01218803FFF7A1FC082071
:100C6000ADF8140003208DF8160018208DF8170039
:100C700005A91F48FFF77FFA1020ADF814000420E3
:100C80008DF8170005A91A48FFF775FA25208DF889
:100C9000000000208DF8010001208DF802008DF881
:100CA00003006846FFF78EFB01940020ADF80800B2
:100CB000ADF80A00ADF80C00ADF810000C20ADF84E
:100CC0000E0001A90B48FFF74DFE012240F225510D
:100CD0000848FFF722FE012240F224410548FFF7B1
:100CE0001CFE01210348FFF7E2FD06B010BD000025
:100CF000000C01400038014000000000000000002E
:100D00000000000000000000000000F800000000EB
:100D1000000000333000000000100C06100C06002C
:100D2000000000000000000040C07840C078400093
:100D3000043F04043F040400007088FC08300000F5
:100D4000001820FF211E0000F008F000E01800004D
:100D500000211C031E211E0000F008887000000006
:100D60001E2123241927211010160E000000000058
:100D70000000000000000000000000E01804020075
:100D8000000000071820400000020418E0000000E6
:100D90000040201807000000404080F080404000E4
:100DA0000202010F01020200000000F0000000003A
:100DB0000101011F0101010000000000000000000E
:100DC00080B0700000000000000000000000000083
:100DD000000101010101010100000000000000000C
:100DE00000303000000000000000000080601804A7
:100DF000006018060100000000E010080810E00084
:100E0000000F102020100F00001010F8000000004C
:100E10000020203F20200000007008080888700093
:100E20000030282422213000003008888848300013
:100E30000018202020110E000000C02010F8000033
:100E400000070424243F240000F8088888080800CC
:100E50000019212020110E0000E0108888180000E1
:100E6000000F112020110E0000380808C8380800B3
:100E70000000003F00000000007088080888700033
:100E8000001C222121221C0000E010080810E000B4
:100E90000000312222110F00000000C0C00000003D
:100EA0000000003030000000000000800000000062
:100EB000000080600000000000008040201008005A
:100EC0000001020408102000404040404040400023
:100ED00004040404040404000008102040800000FE
:100EE0000020100804020100007048080808F00003
:100EF0000000003036010000C030C828E810E000D3
:100F00000718272423140B000000C038E00000005D
:100F1000203C23020227382008F8888888700000C7
:100F2000203F202020110E00C0300808080838009B
:100F3000071820202010080008F808080810E00012
:100F4000203F202020100F0008F88888E8081000B3
:100F5000203F20202320180008F88888E808100087
:100F6000203F200003000000C030080808380000BF
:100F700007182020221E020008F808000008F808C0
:100F8000203F210101213F20000808F80808000047
:100F90000020203F2020000000000808F80808007A
:100FA000C08080807F00000008F888C028180800F2
:100FB000203F20012638200008F80800000000002B
:100FC000203F20202020300008F8F800F8F8080022
:100FD000203F003F003F200008F830C00008F8081C
:100FE000203F200007183F00E01008080810E0002C
:100FF0000F10202020100F0008F808080808F00043
:10100000203F210101010000E01008080810E00065
:101010000F18242438504F0008F8888888887000FA
:10102000203F2000030C302000708808080838009A
:101030000038202121221C00180808F80808180090
:101040000000203F2000000008F808000008F80811
:10105000001F202020201F000878880000C83808C2
:10106000000007380E010000F80800F80008F8003A
:10107000033C0700073C03000818688080681808D4
:1010800020302C03032C30200838C800C838080052
:101090000000203F2000000010080808C8380800A1
:1010A0002038262120201800000000FE0202020045
:1010B0000000007F40404000000C30C000000000F5
:1010C000000000010638C00000020202FE0000001D
:1010D000004040407F0000000000040202020400C3
:1010E0000000000000000000000000000000000000
:1010F00080808080808080800002020400000000E8
:1011000000000000000000000000808080800000DF
:101110000019242222223F2008F8008080000000CD
:10112000003F112020110E00000000808080000090
:10113000000E112020201100000000808088F8009F
:10114000000E112020103F200000808080800000D1
:10115000001F222222221300008080F08888881835
:101160000020203F20200000000080808080800040
:10117000006B94949493600008F8008080800000D5
:10118000203F210000203F200080989800000000B0
:101190000020203F202000000000008098980000E0
:1011A00000C08080807F000008F800008080800000
:1011B000203F24022D302000000808F80000000025
:1011C0000020203F202000008080808080808000E0
:1011D000203F20003F20003F808000808080000072
:1011E000203F210000203F20000080808080000000
:1011F000001F202020201F00808000808000000031
:1012000080FFA12020110E0000000080808080005F
:10121000000E112020A0FF80808080008080800050
:1012200020203F212000010000008080808080007D
:101230000033242424241900008080E080800000F2
:101240000000001F2020000080800000008080003F
:10125000001F202020103F208080800000808080A0
:1012600000010E3008060100808000800080808030
:101270000F300C030C300F00008080008080800055
:101280000020312E0E312000808080000080808080
:1012900080818E7018060100008080808080800030
:1012A0000021302C2221300000000000807C02024E
:1012B00000000000003F404000000000FF00000070
:1012C00000000000FF0000000002027C800000001F
:1012D0000040403F0000000000060101020204043B
:1012E00000000000000000000813000800000020BB
:1012F000240000006C0A00082C13000824000020C1
:10130000140400007C0A000800000000010203042D
:101310000102030406070809020406080000000091
:0C132000006F00630000000000000000EF
:04000005080000ED02
:00000001FF
